:100000008A110A120528000009000730990083169A
:10001000051085100511051283120510051105162E
:10002000E830A0000330A100B7212C30A00001303F
:10003000A100B7213820AC012C080A3C031C34284D
:10004000AD012D083B3C031C2E28BC30A000023023
:10005000A100B7210130AD07031C21281F30830503
:100060000130AC07031C1C281F30830515283728D6
:1000700005145830A0000230A100B721D420572128
:10008000D4205721D42066218D205721912066212C
:10009000AD205721D02057211C2157218D205721D9
:1000A000882057219C206621AD205721D020572140
:1000B0001C2157218D205721882057219C20662103
:1000C000AD205721D02057211C2157218D205721A9
:1000D000882057219C206621982057219320572162
:1000E000EC2057210A215721C6205721B220662132
:1000F000A3219030A0000130A100B7210510080015
:100100007D219021080090217D217D217D21080005
:1001100090217D2190217D21080090217D217D214C
:1001200008007D2108007D217D2190217D2108008E
:10013000902190217D2108007D217D217D217D213F
:1001400008007D217D2108007D21902190219021B2
:10015000080090217D21902108007D2190217D21A2
:100160007D21080090219021080090217D21080028
:1001700090219021902108007D21902190217D21C6
:100180000800902190217D21902108007D2190215F
:100190007D2108007D217D217D210800902108001E
:1001A0007D217D21902108007D217D217D219021CF
:1001B00008007D2190219021080090217D217D2142
:1001C0009021080090217D2190219021080090210C
:1001D00090217D217D210800902190219021902166
:1001E000902108007D2190219021902190210800EC
:1001F0007D217D2190219021902108007D217D216C
:100200007D219021902108007D217D217D217D216E
:10021000902108007D217D217D217D217D21080007
:1002200090217D217D217D217D210800902190213B
:100230007D217D217D2108009021902190217D212B
:100240007D21080090219021902190217D2108009E
:100250007D2190217D2190217D21902108009021F8
:1002600090217D217D219021902108007D217D21FB
:10027000902190217D217D21080090217D217D21EB
:1002800090217D21080090217D217D217D219021DB
:10029000080090217D217D217D217D219021080074
:1002A000051105166430A000A101B7210800051151
:1002B00005166430A000A101B7216430A000A1019F
:1002C000B7216430A000A101B7210800051105166F
:1002D0006430A000A101B7216430A000A101B721C2
:1002E0006430A000A101B7216430A000A101B721B2
:1002F0006430A000A101B7210800051505120530E2
:1003000084000230AA009930A0000230A1004430DD
:10031000A2000030A300F2210511051650210800AB
:1003200005150512053084000230AA009930A0009E
:100330000230A1000E30A2000130A300F22105110D
:1003400005165021080005150512053084000230FD
:10035000AA009930A0000230A100EE30A2000230C5
:10036000A300F2210511051650210800B629A008A6
:100370000319C229C921A0030000000000000000E9
:100380000000B729A10803190800C921A103A0038F
:10039000B7290C30A500A50BCB29000000001230B6
:1003A000A200A20BD829DA21DA21000000000800FF
:1003B000DA21D1290D30A400A40BDC2900000800AB
:1003C0001030A8020001031C013EA902031C080012
:1003D000E9290A30A8020001031C013EA902031CFE
:1003E0000800E9292A0880042008A8002108A9009B
:1003F000E0210130A202031CA3032A098005200882
:10040000A8002108A900E021A208031DF229A308E1
:06041000031DF2290800A3
:02400E00C431BB
:00000001FF
